:100000002500A304C10BE201D10BD30BD50BD70BF9
:10038200D20C02000C0C0600110C2600A4047D0005
:10039200DB0B3D024307CF0B040C3D00FD00F80BC5
:1003A200110CD80B120CD80B220CD80B210C2600E6
:1003B200DB0B7D004607DB0B000C6606010CA40478
:1003C2003E004607DB0B000C6606010C3F009E0157
:1003D2004307DB0B4606EB0B4606DB0BA4043E028F
:1003E2004307CA0BBD021D02040F43067D001D0216
:0E03F2002700040C87000306DA0B0702030A3B
:021FFE000A00D7
:00000001FF
